:0600000000308600072815
:080008009C0A0B11090083168C
:1000100000308600C53081000430850000309A0031
:100020008312A0308B00103085000C3084008001DA
:10003000840A841E1728041E172824222130CE2368
:100040009D002430CE23A0002230CE23A700A200A2
:100050000230CE23AD001E30CE23AF002330CE239E
:100060009B009B181B150430A4002B120510F421D3
:10007000C82093200A21322238281918422805194D
:10008000A80A0800051DA80A080019184A28051D15
:100090004728080005194A28080019185228051988
:1000A0004F280800051D522808009C0177201918C8
:1000B0005C28051961285E28051D61289C18702898
:1000C0005628772077207720A8013D2077207720B9
:1000D0003D207720EC203D208511023028020800C9
:1000E000203089001E088800BE2345201E281A18CB
:1000F00086288611010C7F39031982281E02031CF1
:10010000061108009E08031D061508000611010CC3
:100110007F3903198F281E02031C861108009E08D0
:10012000031D861508001408900015089100160894
:1001300092001708930094019501960197011430DD
:100140008400A520AD20B5200800083098004D207F
:100150005520800D980BA7280800840A4D205520B3
:10016000800D4D205520800D0800840A0430980031
:100170004D205520800C840A4D205520800C98037A
:100180000319C4288403B828800E8403800E080055
:100190002030A8001918DC2813300519173E9800E4
:1001A000A80BD4281914C8280519CC287720EC20CE
:1001B000980BD428851108001330051D173E9800B0
:1001C000A80BE4281910C828051DDC287720EC208E
:1001D000980BE42885110800AB1C072921081E0292
:1001E000031C052903102A0D1B1C2A08323E1B186C
:1001F0000A3E8F00010C8F02031808007D3C031C8F
:1002000003290510080005140800051477289B1819
:1002100005107728851510081402031D2B291108D5
:100220001502031D2B2912081602031D2B29130882
:100230001702031D2B2910081D02031925291B1F56
:100240002B2910082002031D2B29772012081302E6
:100250000319B8292C2908002B161708FE3E03198C
:100260005329FF3E03190613FF3E03198613FF3E71
:1002700003195929FF3E0319A421FF3E03198921BF
:10028000FD3E03195E29FF3E03190617FF3E0319C1
:100290008617FF3E03195629FF3E0319AE21FF3E84
:1002A00003199721D2291208073C7D291208F83E2C
:1002B0007D291208073C031871297D290830160290
:1002C000031C7D2903192B29FD3E03190617FF3E48
:1002D00003198617FE3E0319AE21FF3E031997212D
:1002E000D22903198921FF3E0319A421FE3E0319D7
:1002F0008613FF3E03190613D229130801391A0683
:100300000319D229130801399A002C2201309200D6
:10031000D2299B1E9529AB1E0800A8002230CE23AF
:10032000A700A200AB1228080800851008009B1E39
:10033000A229AB1A0800A8000130A700A200AB1642
:1003400028080800851408001B1DAC299B1CAA293D
:10035000AB1008002B110800051008001B1DB62962
:100360009B1CB429AB1408002B15080005140800C9
:1003700077201208013A031DCD292B18C329FF301D
:10038000A3000430A4002B1876222B18D2292B149A
:100390009A0901309A052C22D2299B18AB142B1CE8
:1003A000D2292B107720F4211208013A0319F129E0
:1003B0001208AA002B19E9290310AA0D9B1FED2989
:1003C00091080319ED29111CAA0A9118ED29AA0A0E
:1003D000ED292B1EED293030AA072A08CE23A100D3
:1003E0000800A1019E0108001B1A162A1A18072AE4
:1003F000061286169E08031986129B1D86162B1A56
:1004000008009118052A061308000617080086122E
:1004100006169E08031906129B1D06162B1A0800C5
:100420009118142A86130800861708001A181E2A25
:10043000061291188616911C8612080086129118D1
:100440000616911C061208002030CE239E00A10043
:100450002530CE239A000800253089001A0888002C
:10046000BE2308002708013C031D392A21089E00ED
:1004700008002B1221081E0203190800A20B080015
:100480002D081E0203184D2AA10803194A2A2D0817
:100490009E004D2A9E01A20A080021081E02031C8C
:1004A000532A9E03542A9E0A2708A2009C01263044
:1004B000CE231E08AE00880B5E2A622AAE07031800
:1004C0009C0A5B2A043088009C0CAE0C9C13880BA1
:1004D000642A9C0803186E2A9C0CAE0C2730CE238D
:1004E0002E080802031C0030A2070800A30B080016
:1004F0007A2A0800FF30A300A40B0800B02AA50048
:10050000A50A0B30AB1BD42BA50B872A0800861637
:100510000616D42386120612D423842A0230A5009C
:100520002F30822A9D221208013A0319922A9D2215
:100530001208013A031D972A0800C82093201008CA
:100540001402031D9D2A11081502031D9D2A12087D
:100550001602031D9D2A13081702031D9D2A080079
:10056000AB1009307F2201307F229222DA23A803C8
:100570000319E12AA8030319E92AA8030319F22A97
:10058000A80303192C2BA8030319402BA803031954
:10059000922BA80303199A2BA8030319712BA80304
:1005A0000319822BA8030319502BA8030319632BEB
:1005B0000430A8020319AA2B10080319B62B8E22A7
:1005C000B52A7F2292222130890010088800BE239C
:1005D000B32A7F22922222308900DA232808880059
:1005E000BE23B32A7F229222DA2389000310890DC9
:1005F00010080319112B10302802031C012B8E2226
:10060000F32A28087F229222DA230310A80DA81FBC
:100610000B2B8E22032B28088800BE2301307F225B
:10062000F32A0630A500CE23A800A5032503CE2378
:10063000A8020310280C880725088900BE2383160A
:100640008818202B8312A50A1E3025020318B32A0E
:10065000A50AA50A2508132B7F229222DA2304304B
:100660002802031C352B8E222D2B2330CE23E7307E
:100670008805A80328188815A8180816BE23B32AC9
:100680007F229222DA2303302802031C492B8E2278
:10069000412B2330CE238812281C8816BE23B32A70
:1006A0007F229222DA2304302802031C5B2B2130A4
:1006B0002802031C5D2B8E22512B2630890028082E
:1006C0008800BE23B32A7F229222DA23A808031DC2
:1006D0006B2B8E22642B2730890028088800BE23CC
:1006E000B32A7F229222DA2305302802031C7A2BB8
:1006F0008E22722B2330CE23F830880528088804F8
:10070000BE23B32A7F229222DA2303302802031C5D
:100710008B2B8E22832B2330CE238813281C881703
:10072000BE23B32A7F229222243089001008880039
:10073000BE23B32A7F229222DA2303302802031C2D
:10074000A32B8E229B2B2330CE230813281C0817A3
:10075000BE23B32A9222DA2303302802031CB22BD1
:100760008E22AA2BAB13281CAB17B32AFF30A30091
:100770000430A40001307F229C211E2883168B1395
:1007800008128811081555308900AA30890088148C
:1007900008118818C92B83128B170800890083164B
:1007A00008148312080808009C019C029C08031D81
:1007B000D62B0800A801901FE02BA80A101FA80A3A
:1007C000901EE62B0330A807101EA807901DEC2BE7
:1007D0000930A807101DA807901CF22B1B30A80792
:0807E000101CA80728080800FE
:02400E00FB3F76
:104200000000000012000000140015001600180045
:104210001A001C001E0020002200250028002B0090
:104220002E00320036003A003E00430048004E00A7
:1042300054005A00600067006E0075007C000000AA
:1042400000002A0003002000A900000010001E004A
:10425000000000000000000000000000000000005E
:104260000000000008000A000C000E001000120000
:10427000150018001B001E002100250029002D003C
:00000001FF
